:020000040000FA
:06000000E73001303A2850
:08000800A000030EA100831209
:1000100005191128831601178312B2308100B1012E
:100020002C2883160113831203140B190310A80D37
:10003000A90DAA0DAB0DAC0DAC16FF302C02031DA3
:100040002C28FA302B02031D2C2832152A08AF0069
:100050002908AE002808AD008B100B11210E83007B
:06006000A00E200E0900B5
:04006600003400342E
:0C007400203084008001840A80300402E7
:10008000031C3C28B82183160C3085058701831298
:10009000850187010730990000309A0010308316DF
:1000A0008E008312603083168F0083120030831617
:1000B00091009F008312C830831681008312313073
:1000C0009000003083168C00831210308B00DC22ED
:1000D00081018E018F010B118B100B108C018B177E
:1000E0007F2032198B20B40B7D280310851903144F
:1000F000BA0DF0303A02031922213D237028640022
:100100003310B10A311F8A28AC01AB01AA01A90141
:10011000A801B101080032110130B7008B13203063
:10012000370783169B001C141A088312A400103092
:10013000370783169B001C141A088312A300A6001D
:100140000230A6060030370783169B001C141A08DD
:100150008312A200A7000130A7068B17331CB62814
:1001600022090339A200A309A409A50924082F0222
:10017000031D1C2923082E02031D1C2922082D0201
:10018000031D1C2901303702031DCB283E18CB2844
:100190003E143F14D32102303702031DD428BE1869
:1001A000D428BE143F14E52103303702031DDD2897
:1001B0003E19DD283E153F14FF2104303702031D90
:1001C000E628BE19E628BE153F141922053037026D
:1001D000031DEF283E1AEF283E163F142B2206304F
:1001E0003702031DF828BE1AF828BE163F143D2218
:1001F00007303702031D01293E1B01293E173F141A
:100200004F2208303702031D0A29BE1B0A29BE17D8
:100210003F14612209303702031D13295E18132988
:100220005E143F1473220A303702031D1C29DE18A6
:100230001C29DE143F148622B70A0B30370203183C
:1002400008008E280130B600B400B500B700850163
:100250008701B2137F20B40B3A29031085190314C8
:10026000BA0DF0303A0203196229B50B3A299630DB
:10027000B5006C21321D2A293211331C44292D0965
:100280000339AD00AE09AF092F1C2A292D08300211
:1002900003192A292D08B0002E1E2A298B1320307D
:1002A0003707BC002F08BB00A32110303707BC0064
:1002B0002E08BB00A32100303707BC002D08BB006F
:1002C000A3218B1785018701B70AB6010B303702CE
:1002D000031C2A29DC220800013037020319AA2254
:1002E000023037020319AF22033037020319B42258
:1002F000043037020319B922053037020319BE2230
:10030000063037020319C322073037020319C82207
:10031000083037020319CD22093037020319D222DF
:100320000A3037020319D72208003F1C08003F108B
:100330001030BC003E08BB00A3213030BC005E087A
:10034000BB00A32108008B133B0883161C159A00E1
:1003500083123C0883169B0055309D00AA309D00F7
:100360009C1464009C18B1291C1183128B1708007F
:10037000831610309B001C141A088312BE008316CB
:1003800030309B001C141A088312DE00FF30C800B6
:10039000CA15CB15CC15CD15CE15CF15D015D11549
:1003A000D215D31508000130BE05FF30DE0511302F
:1003B000C405C0000030C200C6000030C505C10041
:1003C0000030C300C7005F1008000230BE05FF30D8
:1003D000DE054230DF1A0230C405C0000030DF1AEB
:1003E0000030C200C6004030DF1A8030C505C100B1
:1003F0000030DF1A0030C300C7005F10080004306F
:10040000BE05FF30DE050630DF1A8630C405C000A9
:100410000030DF1A0030C200C6004030DF1A8030E2
:10042000C505C1000030DF1A0030C300C7005F10EF
:1004300008000830BE05FF30DE051830C405C000D6
:100440000030C200C6000030C505C1000030C30046
:10045000C7005F1008001030BE05FF30DE053030E9
:10046000C405C0000030C200C6000030C505C10090
:100470000030C300C7005F1008002030BE05FF3009
:10048000DE053030C405C0002030C200C600003098
:10049000C505C1000030C300C7005F100800403030
:1004A000BE05FF30DE050030C405C0000030C200CC
:1004B000C6004030C505C1000030C300C7005F1052
:1004C00008008030BE05FF30DE050030C405C000E6
:1004D0000030C200C6008030C505C1000030C30036
:1004E000C7005F100800FF30BE050130DE05842A1A
:1004F0000030C405C0000030C200C6000030C50591
:10050000C1000030C300C700992A0800FF30BE05B3
:100510000230DE05972A0030C405C0000030C2005A
:10052000C6000030C505C1000030C300C7009F2AC7
:1005300008005F1A08005F16DF12A52A0800DF1AFC
:100540000800DF165F12A52A0800BE18E5213E1933
:10055000FF21080010308506023087060800203091
:100560008506193087060800213085063830870651
:100570000800023085060230870608000030850634
:10058000063087060800003085060630870608001A
:1005900000308506103087060800003085060830D8
:1005A0008706080033308506173087060800333089
:1005B00085062E30870608005F12DF12DE18DF1670
:1005C000DF1E5F163E18D321BE18E5213E19FF211C
:1005D000BE1919223E1A2B22BE1A3D223E1B4F2263
:1005E000BE1B61225E187322DE1886220800B60147
:1005F000B401B5013D1CFF2ABD01BD14012BBD0195
:100600003D143D08B6006400052B062B072B082B74
:10061000092BFF30B51B8500B51F8501B40B032BDB
:10062000B50B032B0310B60CB608031D032B0030CB
:10063000BC003D08BB00A321080005125C1805168C
:10064000DC1C8512DC1885165C1D05105C19051470
:10065000DC1D8510DC1985145C1E87105C1A87145C
:10066000DC1E0711DC1A07155C1F07105C1B071442
:10067000DC1F8712DC1B871608008F08031908008F
:100680008F0178308E00C80F772DC80ADF196F2BC5
:10069000441C6F2B461C602BCA1C512BCA014A15E7
:1006A0007D2B4A1D562BCA01CA157D2BCA1D5B2BFB
:1006B000CA014A167D2B4A1E7D2BCA01CA147D2B06
:1006C0004A1D652BCA014A167D2BCA1D6A2BCA0119
:1006D0004A167D2B4A1E7D2BCA01CA147D2BCA1CCB
:1006E000742BCA014A157D2B4A1D792BCA01CA15E4
:1006F0007D2B4A1E7D2BCA014A15DF19A62BC41C6F
:10070000A62BC61C972BCB1C882BCB014B15B42BCF
:100710004B1D8D2BCB01CB15B42BCB1D922BCB01BD
:100720004B16B42B4B1EB42BCB01CB14B42B4B1D4F
:100730009C2BCB014B16B42BCB1DA12BCB014B1605
:10074000B42B4B1EB42BCB01CB14B42BCB1CAB2B3B
:10075000CB014B15B42B4B1DB02BCB01CB15B42BC0
:100760004B1EB42BCB014B15DF19DD2B441DDD2BAC
:10077000461DCE2BCC1CBF2BCC014C15EB2B4C1D9E
:10078000C42BCC01CC15EB2BCC1DC92BCC014C16AA
:10079000EB2B4C1EEB2BCC01CC14EB2B4C1DD32B99
:1007A000CC014C16EB2BCC1DD82BCC014C16EB2BD3
:1007B0004C1EEB2BCC01CC14EB2BCC1CE22BCC0134
:1007C0004C15EB2B4C1DE72BCC01CC15EB2B4C1E09
:1007D000EB2BCC014C15DF19152CC41D152CC61D97
:1007E000062CCD1CF72BCD014D155F13232C4D1D71
:1007F000FC2BCD01CD15232CCD1D012CCD014D168B
:10080000232C4D1E232CCD01CD14232C4D1D0B2C40
:10081000CD014D16232CCD1D102CCD014D16232CB2
:100820004D1E232CCD01CD14232CCD1C1A2CCD0113
:100830004D15232C4D1D1F2CCD01CD15232C4D1EE8
:10084000232CCD014D15DF194E2C5F1B4E2C441E61
:100850004E2C461E3F2CCE1C302CCE014E155C2C4F
:100860004E1D352CCE01CE155C2CCE1D3A2CCE0162
:100870004E165C2C4E1E5C2CCE01CE145C2C4E1DF4
:10088000442CCE014E165C2CCE1D492CCE014E16AA
:100890005C2C4E1E5C2CCE01CE145C2CCE1C532C3A
:1008A000CE014E155C2C4E1D582CCE01CE155C2C65
:1008B0004E1E5C2CCE014E15DF19852CC41E852CD6
:1008C000C61E762CCF1C672CCF014F15932C4F1DC5
:1008D0006C2CCF01CF15932CCF1D712CCF014F164F
:1008E000932C4F1E932CCF01CF14932C4F1D7B2C98
:1008F000CF014F16932CCF1D802CCF014F16932C78
:100900004F1E932CCF01CF14932CCF1C8A2CCF01D8
:100910004F15932C4F1D8F2CCF01CF15932C4F1EAD
:10092000932CCF014F15DF19BC2C441FBC2C461F44
:10093000AD2CD01C9E2CD0015015CA2C501DA32CC0
:10094000D001D015CA2CD01DA82CD0015016CA2C0D
:10095000501ECA2CD001D014CA2C501DB22CD0016C
:100960005016CA2CD01DB72CD0015016CA2C501EC0
:10097000CA2CD001D014CA2CD01CC12CD0015015C7
:10098000CA2C501DC62CD001D015CA2C501ECA2C02
:10099000D0015015DF19F32CC41FF32CC61FE42C13
:1009A000D11CD52CD1015115012D511DDA2CD101AD
:1009B000D115012DD11DDF2CD1015116012D511E54
:1009C000012DD101D114012D511DE92CD101511658
:1009D000012DD11DEE2CD1015116012D511E012DDD
:1009E000D101D114012DD11CF82CD1015115012DAB
:1009F000511DFD2CD101D115012D511E012DD1010B
:100A00005115451F292D471F1A2DD21C0B2DD20120
:100A10005215DF13372D521D102DD201D215372D4F
:100A2000D21D152DD2015216372D521E372DD2014F
:100A3000D214372D521D1F2DD2015216372DD21D23
:100A4000242DD2015216372D521E372DD201D21429
:100A5000372DD21C2E2DD2015215372D521D332D7C
:100A6000D201D215372D521E372DD2015215DF1B60
:100A7000602DC51F602DC71F512DD31C422DD301E2
:100A800053156E2D531D472DD301D3156E2DD31D38
:100A90004C2DD30153166E2D531E6E2DD301D3143E
:100AA0006E2D531D562DD30153166E2DD31D5B2D68
:100AB000D30153166E2D531E6E2DD301D3146E2DFC
:100AC000D31C652DD30153156E2D531D6A2DD301F3
:100AD000D3156E2D531E6E2DD3015315952140084D
:100AE000C4004108C5005F18DF145F1CDF10480810
:100AF000C9000C304A05031D05120C304B05031DBF
:100B000085120C304C05031D05100C304D05031DDE
:100B100085100C304E05031D87100C304F05031D4A
:100B200007110C305005031D07100C305105031D33
:100B300087120C305205031D07120C305305031D9C
:100B4000871149080E020318D12D12304A05031DE2
:100B5000051612304B05031D851612304C05031D7A
:100B6000051412304D05031D851412304E05031D6A
:100B7000871412304F05031D071512305005031D51
:100B8000071412305105031D871612305205031D3C
:100B9000071612305305031D8715FF30480203194D
:100BA00008008F08031D08007F2049080E02031C5F
:100BB000D12D18304A05031D051206304A05031DC4
:100BC000051618304B05031D851206304B05031D15
:100BD000851618304C05031D051006304C05031D05
:100BE000051418304D05031D851006304D05031DF5
:100BF000851418304E05031D871006304E05031D61
:100C0000871418304F05031D071106304F05031DCB
:100C1000071518305005031D071006305005031D39
:100C2000071418305105031D871206305105031DA6
:100C3000871618305205031D071206305205031D92
:100C4000071618305305031D871106305305031D81
:040C500087150800FC
:084000000C000300060009009A
:02400E00CC33B1
:10420000010078007A007C007E007B0079007F004E
:104210007D007A0078007E007C007D007F007900C0
:104220000200F200F600FA00FE00F200F600FA00CA
:10423000FE00F200F600FA00FE00F200F600FA00BE
:10424000FF00050005000500050009000900090040
:1042500009000D000D000D000D00110011001100EE
:104260000100FF00FF00FF00FF00FF00FF00FF0054
:10427000FF00FF00FF00FF00FF00FF00FF00FF0046
:10428000FF007B00FF00FF00FF00FF00FF00FF00BA
:10429000FF00FF00FF00FF00FF00FF00FF00FF0026
:1042A000FF00FE00FF00FF00FF00FF00FF00FF0017
:1042B000FF00FF00FF00FF00FF00FF00FF00FF0006
:1042C000FF001100FF00FF00FF00FF00FF00FF00E4
:1042D000FF00FF00FF00FF00FF00FF00FF00FF00E6
:1042E000FF00FF00FF00FF00FF00FF00FF00FF00D6
:1042F000FF00FF00FF00FF00FF00FF00FF00DD00E8
:00000001FF
